:020000040000FA
:04080000DBEF06F034
:1008100003B20AEF05F0F2B428EF05F09EB030EF16
:1008200005F09EB238EF05F0F2A81AEF04F0F2B22C
:100830001CEF04F08AEF06F0CD90F2929EA026EF16
:1008400004F00101533F26EF04F0542BAEC1B2F186
:10085000AFC1B3F1B0C1B4F1B1C1B5F1AAC1AEF14C
:10086000ABC1AFF1ACC1B0F1ADC1B1F1A6C1AAF15C
:10087000A7C1ABF1A8C1ACF1A9C1ADF1A2C1A6F16C
:10088000A3C1A7F1A4C1A8F1A5C1A9F19EC1A2F17C
:100890009FC1A3F1A0C1A4F1A1C1A5F19AC19EF18C
:1008A0009BC19FF19CC1A0F19DC1A1F196C19AF19C
:1008B00097C19BF198C19CF199C19DF1CECF96F162
:1008C000CFCF97F153C198F154C199F1CF6ACE6A55
:1008D0000101536B546B9E90CD800FBC0F8E0FBAED
:1008E00075EF04F00F8A8AEF06F00F8C0FBEB1EFA0
:1008F00004F096C19AF197C19BF198C19CF199C1FE
:100900009DF19AC19EF19BC19FF19CC1A0F19DC137
:10091000A1F19EC1A2F19FC1A3F1A0C1A4F1A1C107
:10092000A5F1A2C1A6F1A3C1A7F1A4C1A8F1A5C1D7
:10093000A9F1A6C1AAF1A7C1ABF1A8C1ACF1A9C1A7
:10094000ADF1AAC1AEF1ABC1AFF1ACC1B0F1ADC177
:10095000B1F1AEC1B2F1AFC1B3F1B0C1B4F1B1C147
:10096000B5F101015E6B5F6B606B616B96515E2749
:1009700097515F2398516023995161239A515E27C3
:100980009B515F239C5160239D5161239E515E27A3
:100990009F515F23A0516023A1516123A2515E2783
:1009A000A3515F23A4516023A5516123A6515E2763
:1009B000A7515F23A8516023A9516123AA515E2743
:1009C000AB515F23AC516023AD516123AE515E2723
:1009D000AF515F23B0516023B1516123B2515E2703
:1009E000B3515F23B4516023B5516123D890010105
:1009F000613360335F335E33D8900101613360331C
:100A00005F335E33D8900101613360335F335E330F
:100A10008AEF06F00392ABB2AB98AB88030103EE0A
:100A200000F080517F0BE92604C0EFFF802B81513D
:100A3000805D700BD8A48B8200008051815D700BAB
:100A4000D8A48B9281518019D8B407908AEF06F010
:100A5000F2940101453F8AEF06F0462B8AEF06F03B
:100A60009E900101533F8AEF06F0542B8AEF06F067
:100A70009E92C3CF55F1C4CF56F1C28207B4A3EF03
:100A800005F047C14BF148C14CF149C14DF14AC194
:100A90004EF15EC162F15FC163F160C164F161C199
:100AA00065F196C1B6F197C1B7F198C1B8F199C196
:100AB000B9F19AC1BAF19BC1BBF19CC1BCF19DC116
:100AC000BDF19EC1BEF19FC1BFF1A0C1C0F1A1C1E6
:100AD000C1F1A2C1C2F1A3C1C3F1A4C1C4F1A5C1B6
:100AE000C5F1A6C1C6F1A7C1C7F1A8C1C8F1A9C186
:100AF000C9F1AAC1CAF1ABC1CBF1ACC1CCF1ADC156
:100B0000CDF1AEC1CEF1AFC1CFF1B0C1D0F1B1C125
:100B1000D1F1B2C1D2F1B3C1D3F1B4C1D4F1B5C1F5
:100B2000D5F1010155515B2756515C23E86A5D23DD
:100B30000E2EA3EF05F05CC157F15DC158F15B6B60
:100B40005C6B5D6B078E0201002F8AEF06F03C0E96
:100B5000006F00C10CF101C10DF102C10EF103C122
:100B60000FF104C110F105C111F106C112F107C165
:100B700013F108C114F109C115F10AC116F10BC135
:100B800017F134C135F101018A67CEEF05F08B67AB
:100B9000CEEF05F08C67CEEF05F08D67D2EF05F054
:100BA00002EF06F08EC100F18FC101F190C102F198
:100BB00091C103F10101010E046F000E056F000EDB
:100BC000066F000E076F5EEC15F000C18EF101C1DB
:100BD0008FF102C190F103C191F10067F7EF05F0C9
:100BE0000167F7EF05F00267F7EF05F0036702EF23
:100BF00006F08AC18EF18BC18FF18CC190F18DC14D
:100C000091F10F80D57ED5BE69D0D6CF47F1D7CF31
:100C100048F145C149F1E86AE8CF4AF1109047C16F
:100C200000F148C101F149C102F14AC103F10101DA
:100C30000A0E046F000E056F000E066F000E076FA0
:100C40005EEC15F003AF1080010154A734EF06F0FD
:100C50000F9A0F9C0F9E0101000E5E6F600E5F6F7A
:100C60003D0E606F080E616F010147BF44EF06F053
:100C7000486744EF06F0496744EF06F04A6744EFDF
:100C800006F0F28869EF06F0F2985E6B5F6B606BBE
:100C9000616B966B976B986B996B9A6B9B6B9C6B6C
:100CA0009D6B9E6B9F6BA06BA16BA26BA36BA46BE8
:100CB000A56BA66BA76BA86BA96BAA6BAB6BAC6B98
:100CC000AD6BAE6BAF6BB06BB16BB26BB36BB46B48
:100CD000B56BD76AD66A0101456B466B0CC100F152
:100CE0000DC101F10EC102F10FC103F110C104F1F8
:100CF00011C105F112C106F113C107F114C108F1C8
:100D000015C109F116C10AF117C10BF135C134F152
:100D10008AEF06F002C0E0FF005001C0D8FF1000CB
:100D2000A6B290EF06F00CC0A9FF0BC0A8FFA69ECC
:100D3000A69CA684F29E550EA76EAA0EA76EA6824A
:100D4000F28EA694A6B2A2EF06F00C2A1200A96EAB
:100D5000A69EA69CA680A8500C2A120004012C0E68
:100D6000826F6EEC08F059EC16F00C50A7EC06F010
:100D7000E8CF00F10C50A7EC06F0E8CF01F101AF8D
:100D8000C7EF06F00101FF0E026FFF0E036FFCECD0
:100D900015F02967D3EF06F00401200E826F6EEC88
:100DA00008F0D8EF06F004012D0E826F6EEC08F00B
:100DB00026EC14F01200076A0F6A106A0F010E0E7B
:100DC000C16E860EC06E030EC26E0F01896A110ECF
:100DD000926E080E8A6EF10E936E8B6A800E946E80
:100DE000F18E0E6A01015B6B5C6B5D6B576B586B30
:100DF000F29A0101476B486B496B4A6B4B6B4C6B2A
:100E00004D6B4E6B4F6B506B516B526B456B466B22
:100E1000D76AD66A0F01280ED56EF28A9D90B00E61
:100E2000CD6E01015E6B5F6B606B616B626B636BC0
:100E3000646B656B666B676B686B696B536B546B4C
:100E4000CF6ACE6A0F9A0F9C0F9E9D80760ECA6E57
:100E50009D8202013C0E006FCC6A160EA7EC06F0D4
:100E6000E8CF00F1170EA7EC06F0E8CF01F1180E5D
:100E7000A7EC06F0E8CF02F1190EA7EC06F0E8CFD8
:100E800003F1010103AF5FEF07F059EC16F0160E06
:100E90000C6E00C10BF090EC06F0170E0C6E01C149
:100EA0000BF090EC06F0180E0C6E02C10BF090ECFB
:100EB00006F0190E0C6E03C10BF090EC06F000C1A9
:100EC0008AF101C18BF102C18CF103C18DF100C126
:100ED0008EF101C18FF102C190F103C191F11A0E9F
:100EE000A7EC06F0E8CF00F11B0EA7EC06F0E8CF68
:100EF00001F11C0EA7EC06F0E8CF02F11D0EA7ECE5
:100F000006F0E8CF03F1010103AFB5EF07F059ECAC
:100F100016F01A0E0C6E00C10BF090EC06F01B0ED2
:100F20000C6E01C10BF090EC06F01C0E0C6E02C1B1
:100F30000BF090EC06F01D0E0C6E03C10BF090EC64
:100F400006F01A0EA7EC06F0E8CF00F11B0EA7EC96
:100F500006F0E8CF01F11C0EA7EC06F0E8CF02F195
:100F60001D0EA7EC06F0E8CF03F100C192F101C11C
:100F700093F102C194F103C195F1240EAC6E900E71
:100F8000AB6E240EAC6E080EB86E000EB06E1F0E67
:100F9000AF6E0401806B816B0F01900EAB6E0F0181
:100FA0009D8A0301806B816BC26B8B92079000015D
:100FB000F28EF28C07B0D3EF12F00FB0B2EF0DF05B
:100FC0000301805181197F0BD8B4D3EF12F013EED7
:100FD00000F081517F0BE126812BE7CFE8FFE00B8A
:100FE000D8B4D3EF12F023EE82F0C2513F0BD926D2
:100FF000E7CFDFFFC22BDF50780AD8A4D3EF12F07F
:1010000007808EC100F18FC101F190C102F191C141
:1010100003F10101040E046F000E056F000E066F50
:10102000000E076F5EEC15F000AF20EF08F0010135
:10103000030E8E6F000E8F6F000E906F000E916F7B
:1010400003018251720AD8B4B2EF0DF08251520AF4
:10105000D8B4B2EF0DF08251750AD8B4B2EF0DF0EA
:101060008251630AD8B48DEF0FF08251690AD8B467
:101070006DEF0AF082517A0AD8B480EF0BF08251FA
:10108000490AD8B40CEF0AF08251500AD8B42AEFBA
:1010900009F08251700AD8B46DEF09F08251540AF8
:1010A000D8B498EF09F08251740AD8B4DEEF09F091
:1010B00082516D0AD8B482EF08F082514D0AD8B43B
:1010C0009BEF08F08251730AD8B4E2EF0CF0825122
:1010D000530AD8B447EF0DF0C4EF0FF0040114EE3B
:1010E00000F080517F0BE12682C4E7FF802B1200C5
:1010F00004010D0E826F6EEC08F00A0E826F6EEC2A
:1011000008F0120004016D0E826F6EEC08F003010E
:101110008351300AD8B4DAEF08F003018351310A61
:10112000D8B4EDEF08F003018351320AD8B400EFD0
:1011300009F0C4EF0FF004014D0E826F6EEC08F061
:101140009AEC16F084C331F185C332F186C333F1D2
:101150000101296BA7EC16F01EEC16F00301835178
:10116000300AD8B4C2EF08F003018351310AD8B471
:10117000CAEF08F003018351320AD8B4D2EF08F065
:10118000C4EF0FF0FD0E0C6E00C10BF090EC06F0FA
:10119000DAEF08F0FE0E0C6E00C10BF090EC06F0DA
:1011A000EDEF08F0FF0E0C6E00C10BF090EC06F0B6
:1011B00000EF09F00401300E826F6EEC08F00401BC
:1011C0002C0E826F6EEC08F059EC16F0FD0EA7ECB9
:1011D00006F0E8CF00F111EF09F00401310E826F43
:1011E0006EEC08F004012C0E826F6EEC08F059ECE6
:1011F00016F0FE0EA7EC06F0E8CF00F111EF09F0B3
:101200000401320E826F6EEC08F059EC16F0040106
:101210002C0E826F6EEC08F0FF0EA7EC06F0E8CF04
:1012200000F1FCEC15F031C182F40401300E82278C
:101230006EEC08F032C182F40401300E82276EECAD
:1012400008F033C182F40401300E82276EEC08F0FE
:10125000C2EF0FF083C32AF184C32BF185C32CF1B5
:1012600086C32DF187C32EF188C32FF189C330F1D6
:101270008AC331F18BC332F18CC333F10101A7EC86
:1012800016F01EEC16F0160E0C6E00C10BF090EC72
:1012900006F0170E0C6E01C10BF090EC06F0180E64
:1012A0000C6E02C10BF090EC06F0190E0C6E03C12F
:1012B0000BF090EC06F000C18AF101C18BF102C184
:1012C0008CF103C18DF100C18EF101C18FF102C11A
:1012D00090F103C191F10CEF0AF083C32AF184C3AA
:1012E0002BF185C32CF186C32DF187C32EF188C362
:1012F0002FF189C330F18AC331F18BC332F18CC332
:1013000033F10101A7EC16F01EEC16F000C18AF1D2
:1013100001C18BF102C18CF103C18DF100C18EF1CD
:1013200001C18FF102C190F103C191F10CEF0AF0FC
:1013300083C32AF184C32BF185C32CF186C32DF11D
:1013400087C32EF188C32FF189C330F18AC331F1ED
:101350008CC332F18DC333F10101A7EC16F01EEC02
:1013600016F00101000E046F000E056F010E066FEE
:10137000000E076F6FEC15F01A0E0C6E00C10BF02B
:1013800090EC06F01B0E0C6E01C10BF090EC06F019
:101390001C0E0C6E02C10BF090EC06F01D0E0C6ED4
:1013A00003C10BF090EC06F000C192F101C193F182
:1013B00002C194F103C195F10CEF0AF083C32AF145
:1013C00084C32BF185C32CF186C32DF187C32EF185
:1013D00088C32FF189C330F18AC331F18CC332F154
:1013E0008DC333F10101A7EC16F01EEC16F00101DC
:1013F000000E046F000E056F010E066F000E076FE2
:101400006FEC15F000C192F101C193F102C194F1AA
:1014100003C195F10CEF0AF0160EA7EC06F0E8CF29
:1014200000F1170EA7EC06F0E8CF01F1180EA7ECBB
:1014300006F0E8CF02F1190EA7EC06F0E8CF03F1B1
:10144000FCEC15F0DFEC13F00401730E826F6EEC10
:1014500008F004012C0E826F6EEC08F08AC100F1D6
:101460008BC101F18CC102F18DC103F1FCEC15F0CF
:10147000DFEC13F00401730E826F6EEC08F00401D0
:101480002C0E826F6EEC08F01A0EA7EC06F0E8CF77
:1014900000F11B0EA7EC06F0E8CF01F11C0EA7EC43
:1014A00006F0E8CF02F11D0EA7EC06F0E8CF03F13D
:1014B000DFEC0FF004012C0E826F6EEC08F092C18D
:1014C00000F193C101F194C102F195C103F1DFEC88
:1014D0000FF078EC08F0C4EF0FF00401690E826F92
:1014E0006EEC08F004012C0E826F6EEC08F0010126
:1014F000040E006F000E016F000E026F000E036FEE
:10150000FCEC15F02CC182F40401300E82276EEC45
:1015100008F02DC182F40401300E82276EEC08F031
:101520002EC182F40401300E82276EEC08F02FC128
:1015300082F40401300E82276EEC08F030C182F490
:101540000401300E82276EEC08F031C182F40401F0
:10155000300E82276EEC08F032C182F40401300EA6
:1015600082276EEC08F033C182F40401300E82272A
:101570006EEC08F004012C0E826F6EEC08F0010195
:10158000030E006F000E016F000E026F000E036F5E
:10159000FCEC15F02CC182F40401300E82276EECB5
:1015A00008F02DC182F40401300E82276EEC08F0A1
:1015B0002EC182F40401300E82276EEC08F02FC198
:1015C00082F40401300E82276EEC08F030C182F400
:1015D0000401300E82276EEC08F031C182F4040160
:1015E000300E82276EEC08F032C182F40401300E16
:1015F00082276EEC08F033C182F40401300E82279A
:101600006EEC08F004012C0E826F6EEC08F0010104
:10161000240E006F000E016F000E026F000E036FAC
:10162000FCEC15F02CC182F40401300E82276EEC24
:1016300008F02DC182F40401300E82276EEC08F010
:101640002EC182F40401300E82276EEC08F02FC107
:1016500082F40401300E82276EEC08F030C182F46F
:101660000401300E82276EEC08F031C182F40401CF
:10167000300E82276EEC08F032C182F40401300E85
:1016800082276EEC08F033C182F40401300E822709
:101690006EEC08F004012C0E826F6EEC08F0200E48
:1016A000F86EF76AF66A04010900F5CF82F46EEC71
:1016B00008F00900F5CF82F46EEC08F00900F5CFD0
:1016C00082F46EEC08F00900F5CF82F46EEC08F0BD
:1016D0000900F5CF82F46EEC08F00900F5CF82F432
:1016E0006EEC08F00900F5CF82F46EEC08F009000A
:1016F000F5CF82F46EEC08F078EC08F0C4EF0FF050
:101700008351630AD8A4C4EF0FF08451610AD8A4AE
:10171000C4EF0FF085516C0AD8A4C4EF0FF08651C6
:10172000410A42E08651440A1BE08651420AD8B47D
:10173000E7EF0BF08651350AD8B44EEF11F0865121
:10174000360AD8B4A3EF11F08651370AD8B40CEF9B
:1017500012F08651380AD8B46AEF12F0C4EF0FF0D5
:101760000798079A04017A0E826F6EEC08F0040164
:10177000780E826F6EEC08F00401640E826F6EECDE
:1017800008F081A8CBEF0BF00401550E826F6EECD0
:1017900008F0D0EF0BF004014C0E826F6EEC08F0F5
:1017A00078EC08F0C4EF0FF00788079A04017A0E6E
:1017B000826F6EEC08F00401410E826F6EEC08F04F
:1017C0000401610E826F6EEC08F0C1EF0BF0079818
:1017D000078A04017A0E826F6EEC08F00401420E53
:1017E000826F6EEC08F00401610E826F6EEC08F0FF
:1017F000C1EF0BF00101666705EF0CF0676705EFBD
:101800000CF0686705EF0CF069671DEF0CF04F678F
:1018100011EF0CF0506711EF0CF0516711EF0CF065
:1018200052671DEF0CF00101000E006F000E016FFA
:10183000000E026F000E036F12000101620E046FB2
:10184000010E056F000E066F000E076F66C100F1F6
:1018500067C101F168C102F169C103F15EEC15F0E5
:1018600003BFA1EF0CF00101000E046FA80E056F7D
:10187000550E066F020E076F66C100F167C101F1D8
:1018800068C102F169C103F166C186F167C187F1E0
:1018900068C188F169C189F15EEC15F003BF5AEFA8
:1018A0000CF00101000E866FA80E876F550E886F31
:1018B000020E896F0E0EA7EC06F0E8CF18F10F0E9E
:1018C000A7EC06F0E8CF19F1100EA7EC06F0E8CF70
:1018D0001AF1110EA7EC06F0E8CF1BF1A7EC14F0FB
:1018E00086C104F187C105F188C106F189C107F1FC
:1018F0005EEC15F007826BEC14F0A7EC14F0079285
:101900006BEC14F086C100F187C101F188C102F1CE
:1019100089C103F107926BEC14F0CC0E046FE00E5A
:10192000056F870E066F050E076F5EEC15F000C1A0
:1019300018F101C119F102C11AF103C11BF1D9EF6C
:101940000CF00101800E006F1A0E016F060E026F7F
:10195000000E036F4FC104F150C105F151C106F1F2
:1019600052C107F15EEC15F003AFBAEF0CF059EC81
:1019700016F012000E0EA7EC06F0E8CF18F10F0ECD
:10198000A7EC06F0E8CF19F1100EA7EC06F0E8CFAF
:101990001AF1110EA7EC06F0E8CF1BF14FC100F1D0
:1019A00050C101F151C102F152C103F107826BEC48
:1019B00014F018C100F119C101F11AC102F11BC1E3
:1019C00003F112000401730E826F6EEC08F0040143
:1019D0002C0E826F6EEC08F0078462C166F163C161
:1019E00067F164C168F165C169F14BC14FF14CC148
:1019F00050F14DC151F14EC152F157C159F158C189
:101A00005AF1079408EC0DF078EC08F0C4EF0FF0F1
:101A100066C100F167C101F168C102F169C103F15A
:101A20000101FCEC15F0DFEC13F00401630E826F92
:101A30006EEC08F004012C0E826F6EEC08F04FC1C2
:101A400000F150C101F151C102F152C103F1010194
:101A5000FCEC15F0DFEC13F00401660E826F6EEC07
:101A600008F004012C0E826F6EEC08F059EC16F0B1
:101A700059C100F15AC101F10101FCEC15F0DFEC94
:101A800013F00401740E826F6EEC08F012001082E5
:101A90000401530E826F6EEC08F004012C0E826F6D
:101AA0006EEC08F083C32AF184C32BF185C32CF1BB
:101AB00086C32DF187C32EF188C32FF189C330F17E
:101AC0008AC331F18BC332F18CC333F10101A7EC2E
:101AD00016F01EEC16F000C166F101C167F102C1FB
:101AE00068F103C169F18EC32AF18FC32BF190C352
:101AF0002CF191C32DF192C32EF193C32FF194C316
:101B000030F195C331F196C332F197C333F101013E
:101B1000A7EC16F01EEC16F000C14FF101C150F118
:101B200002C151F103C152F19AEC16F099C32FF1A1
:101B30009AC330F19BC331F19CC332F19DC333F1A1
:101B40000101A7EC16F01EEC16F000C159F101C11D
:101B50005AF108EC0DF004012C0E826F6EEC08F0C7
:101B6000B9EF0DF08251520A03E10F82B9EF0DF087
:101B70000F928251750A03E11084C0EF0DF01094AA
:101B80008251550A03E11086C7EF0DF010960784C5
:101B900010B224EF0EF010A410EF0EF0B6C166F1F3
:101BA000B7C167F1B8C168F1B9C169F1BAC16AF1E9
:101BB000BBC16BF1BCC16CF1BDC16DF1BEC16EF1B9
:101BC000BFC16FF1C0C170F1C1C171F1C2C172F189
:101BD000C3C173F1C4C174F1C5C175F1C6C176F159
:101BE000C7C177F1C8C178F1C9C179F1CAC17AF129
:101BF000CBC17BF1CCC17CF1CDC17DF1CEC17EF1F9
:101C0000CFC17FF1D0C180F1D1C181F1D2C182F1C8
:101C1000D3C183F1D4C184F1D5C185F118EF0EF0A1
:101C200062C166F163C167F164C168F165C169F1C0
:101C30004BC14FF14CC150F14DC151F14EC152F168
:101C400057C159F158C15AF107940FA046EF0EF051
:101C50000101926733EF0EF0936733EF0EF0946754
:101C600033EF0EF0956737EF0EF046EF0EF0FAEC1B
:101C70000BF092C104F193C105F194C106F195C135
:101C800007F15EEC15F003BF8AEF0FF0FAEC0BF0F2
:101C90000101000E046F000E056F010E066F000EAD
:101CA000076F8FEC15F010A45DEF0EF00401750EB8
:101CB000826F6EEC08F062EF0EF00401720E826F1C
:101CC0006EEC08F004012C0E826F6EEC08F0FCEC58
:101CD00015F0296771EF0EF00401200E826F74EF8A
:101CE0000EF004012D0E826F6EEC08F030C182F40C
:101CF0000401300E82276EEC08F031C182F4040139
:101D0000300E82276EEC08F004012E0E826F6EEC0E
:101D100008F032C182F40401300E82276EEC08F024
:101D200033C182F40401300E82276EEC08F0040106
:101D30006D0E826F6EEC08F004012C0E826F6EEC5B
:101D400008F04FC100F150C101F151C102F152C17F
:101D500003F10101FCEC15F0DFEC13F00401480E77
:101D6000826F6EEC08F004017A0E826F6EEC08F060
:101D700004012C0E826F6EEC08F066C100F167C1A1
:101D800001F168C102F169C103F10101FCEC15F038
:101D9000DFEC13F00401630E826F6EEC08F00401B7
:101DA0002C0E826F6EEC08F066C100F167C101F184
:101DB00068C102F169C103F101010A0E046F000E4E
:101DC000056F000E066F000E076F6FEC15F0000E2A
:101DD000046F120E056F000E066F000E076F8FEC7A
:101DE00015F0FCEC15F02AC182F40401300E8227B4
:101DF0006EEC08F02BC182F40401300E82276EECE9
:101E000008F02CC182F40401300E82276EEC08F039
:101E10002DC182F40401300E82276EEC08F02EC131
:101E200082F40401300E82276EEC08F02FC182F498
:101E30000401300E82276EEC08F030C182F40401F8
:101E4000300E82276EEC08F004012E0E826F6EECCD
:101E500008F031C182F40401300E82276EEC08F0E4
:101E600032C182F40401300E82276EEC08F033C1D7
:101E700082F40401300E82276EEC08F00401730E28
:101E8000826F6EEC08F004012C0E826F6EEC08F08D
:101E900059EC16F059C100F15AC101F1EEEC10F005
:101EA0000FB256EF0FF00FA088EF0FF004012C0EC9
:101EB000826F6EEC08F0200EF86EF76AF66A040185
:101EC0000900F5CF82F46EEC08F00900F5CF82F43A
:101ED0006EEC08F00900F5CF82F46EEC08F0090012
:101EE000F5CF82F46EEC08F00900F5CF82F46EECC9
:101EF00008F00900F5CF82F46EEC08F00900F5CF88
:101F000082F46EEC08F00900F5CF82F46EEC08F074
:101F100078EC08F00F90C4EF0FF00401630E826FAD
:101F20006EEC08F004012C0E826F6EEC08F0CAEC27
:101F30000FF004012C0E826F6EEC08F03DEC10F0F7
:101F400004012C0E826F6EEC08F0B9EC10F0040165
:101F50002C0E826F6EEC08F00101F80E006FCD0EB2
:101F6000016F660E026F030E036FDFEC0FF00401CA
:101F70002C0E826F6EEC08F0CFEC10F078EC08F0CD
:101F8000C4EF0FF078EC08F00301C26B07901092D9
:101F9000D3EF12F0D8900E0EA7EC06F0E8CF00F1C8
:101FA0000F0EA7EC06F0E8CF01F1100EA7EC06F03B
:101FB000E8CF02F1110EA7EC06F0E8CF03F1010122
:101FC000000E046F000E056F010E066F000E076F06
:101FD0008FEC15F0FCEC15F02AC182F40401300EF0
:101FE00082276EEC08F02BC182F40401300E8227A8
:101FF0006EEC08F02CC182F40401300E82276EECE6
:1020000008F02DC182F40401300E82276EEC08F036
:102010002EC182F40401300E82276EEC08F02FC12D
:1020200082F40401300E82276EEC08F030C182F495
:102030000401300E82276EEC08F031C182F40401F5
:10204000300E82276EEC08F004012E0E826F6EECCB
:1020500008F032C182F40401300E82276EEC08F0E1
:1020600033C182F40401300E82276EEC08F00401C3
:102070006D0E826F6EEC08F01200120EA7EC06F0E7
:10208000E8CF00F1130EA7EC06F0E8CF01F1140E33
:10209000A7EC06F0E8CF02F1150EA7EC06F0E8CFAA
:1020A00003F101010A0E046F000E056F000E066FAA
:1020B000000E076F6FEC15F0000E046F120E056F27
:1020C000000E066F000E076F8FEC15F0FCEC15F09C
:1020D0002AC182F40401300E82276EEC08F02BC175
:1020E00082F40401300E82276EEC08F02CC182F4D9
:1020F0000401300E82276EEC08F02DC182F4040139
:10210000300E82276EEC08F02EC182F40401300EEE
:1021100082276EEC08F02FC182F40401300E822772
:102120006EEC08F030C182F40401300E82276EECB0
:1021300008F004012E0E826F6EEC08F031C182F4BB
:102140000401300E82276EEC08F032C182F40401E3
:10215000300E82276EEC08F033C182F40401300E99
:1021600082276EEC08F00401730E826F6EEC08F0AB
:1021700012000A0EA7EC06F0E8CF00F10B0EA7EC58
:1021800006F0E8CF01F10C0EA7EC06F0E8CF02F163
:102190000D0EA7EC06F0E8CF03F1EEEF10F0060EFF
:1021A000A7EC06F0E8CF00F1070EA7EC06F0E8CFA9
:1021B00001F1080EA7EC06F0E8CF02F1090EA7EC3A
:1021C00006F0E8CF03F1EEEF10F0010159EC16F044
:1021D000078457C100F158C101F107940101E80ECD
:1021E000046F800E056F000E066F000E076F6FEC18
:1021F00015F0000E046F040E056F000E066F000E42
:10220000076F8FEC15F0880E046F130E056F000E2C
:10221000066F000E076F5EEC15F00A0E046F000EDD
:10222000056F000E066F000E076F8FEC15F0FCECCB
:1022300015F00101296722EF11F00401200E826FD1
:1022400025EF11F004012D0E826F6EEC08F030C105
:1022500082F40401300E82276EEC08F031C182F462
:102260000401300E82276EEC08F032C182F40401C2
:10227000300E82276EEC08F004012E0E826F6EEC99
:1022800008F033C182F40401300E82276EEC08F0AE
:102290000401430E826F6EEC08F0120087C32AF12E
:1022A00088C32BF189C32CF18AC32DF18BC32EF186
:1022B0008CC32FF18DC330F18EC331F190C332F155
:1022C00091C333F10101296BA7EC16F01EEC16F057
:1022D0000101000E046F000E056F010E066F000E67
:1022E000076F6FEC15F00E0E0C6E00C10BF090EC4A
:1022F00006F00F0E0C6E01C10BF090EC06F0100E04
:102300000C6E02C10BF090EC06F0110E0C6E03C1C6
:102310000BF090EC06F004017A0E826F6EEC08F080
:1023200004012C0E826F6EEC08F00401350E826FF2
:102330006EEC08F004012C0E826F6EEC08F0CAEC13
:102340000FF0D0EF0BF087C32AF188C32BF189C3BC
:102350002CF18AC32DF18BC32EF18CC32FF18DC3C9
:1023600030F18EC331F190C332F191C333F10101E9
:10237000296BA7EC16F01EEC16F0880E046F130EF6
:10238000056F000E066F000E076F63EC15F0000E70
:10239000046F040E056F000E066F000E076F6FECE2
:1023A00015F00101E80E046F800E056F000E066F38
:1023B000000E076F8FEC15F00A0E0C6E00C10BF0CB
:1023C00090EC06F00B0E0C6E01C10BF090EC06F0D9
:1023D0000C0E0C6E02C10BF090EC06F00D0E0C6EA4
:1023E00003C10BF090EC06F004017A0E826F6EECE4
:1023F00008F004012C0E826F6EEC08F00401360E1A
:10240000826F6EEC08F004012C0E826F6EEC08F007
:10241000B9EC10F0D0EF0BF087C32AF188C32BF191
:1024200089C32CF18AC32DF18BC32EF18CC32FF1FC
:102430008DC330F18FC331F190C332F191C333F1C9
:102440000101A7EC16F01EEC16F0000E046F120E40
:10245000056F000E066F000E076F6FEC15F001019F
:102460000A0E046F000E056F000E066F000E076F58
:102470008FEC15F0120E0C6E00C10BF090EC06F014
:10248000130E0C6E01C10BF090EC06F0140E0C6EE6
:1024900002C10BF090EC06F0150E0C6E03C10BF0B0
:1024A00090EC06F004017A0E826F6EEC08F00401E5
:1024B0002C0E826F6EEC08F00401370E826F6EEC0A
:1024C00008F004012C0E826F6EEC08F03DEC10F069
:1024D000D0EF0BF087C32AF188C32BF189C32CF10D
:1024E0008AC32DF18BC32EF18CC32FF18DC330F134
:1024F0008EC331F190C332F191C333F10101296BE5
:10250000A7EC16F01EEC16F0880E046F130E056F84
:10251000000E066F000E076F63EC15F0000E046FDF
:10252000040E056F000E066F000E076F6FEC15F0BE
:102530000101E80E046F800E056F000E066F000E9D
:10254000076F8FEC15F0060E0C6E00C10BF090ECCF
:1025500006F0070E0C6E01C10BF090EC06F0080EB1
:102560000C6E02C10BF090EC06F0090E0C6E03C16C
:102570000BF090EC06F004017A0E826F6EEC08F01E
:1025800004012C0E826F6EEC08F00401380E826F8D
:102590006EEC08F004012C0E826F6EEC08F0CFECAC
:1025A00010F0D0EF0BF081A891EF13F007A84AEFDD
:1025B00013F00101800E006F1A0E016F060E026FFC
:1025C000000E036F4BC104F14CC105F14DC106F182
:1025D0004EC107F15EEC15F003BF91EF13F0D9EC9B
:1025E00013F04BC100F14CC101F14DC102F14EC1DC
:1025F00003F107826BEC14F018C104F119C105F165
:102600001AC106F11BC107F1F80E006FCD0E016F64
:10261000660E026F030E036F5EEC15F00E0E0C6E6D
:1026200000C10BF090EC06F00F0E0C6E01C10BF028
:1026300090EC06F0100E0C6E02C10BF090EC06F060
:10264000110E0C6E03C10BF090EC06F00784010133
:1026500059EC16F057C100F158C101F107940A0E68
:102660000C6E00C10BF090EC06F00B0E0C6E01C16D
:102670000BF090EC06F00C0E0C6E02C10BF090EC1F
:1026800006F00D0E0C6E03C10BF090EC06F00798EF
:1026900091EF13F007AA91EF13F00784010159ECB1
:1026A00016F057C100F158C101F10794060E0C6EE7
:1026B00000C10BF090EC06F0070E0C6E01C10BF0A0
:1026C00090EC06F0080E0C6E02C10BF090EC06F0D8
:1026D000090E0C6E03C10BF090EC06F0078462C18A
:1026E00000F163C101F164C102F165C103F1079416
:1026F000120E0C6E00C10BF090EC06F0130E0C6E77
:1027000001C10BF090EC06F0140E0C6E02C10BF040
:1027100090EC06F0150E0C6E03C10BF090EC06F079
:10272000079A0401805181197F0B0BE09EA809D004
:1027300014EE00F081517F0BE126E750812B0F0151
:10274000AD6EDAEF07F018C100F119C101F11AC13D
:1027500002F11BC103F1000E046F000E056F010EA4
:10276000066F000E076F8FEC15F029A1CEEF13F066
:102770002051D8B4CEEF13F018C100F119C101F106
:102780001AC102F11BC103F1000E046F000E056FA8
:102790000A0E066F000E076F8FEC15F01200010194
:1027A000045100130551011306510213075103137D
:1027B00012000101186B196B1A6B1B6B12002AC1F6
:1027C00082F40401300E82276EEC08F02BC182F4F3
:1027D0000401300E82276EEC08F02CC182F4040153
:1027E000300E82276EEC08F02DC182F40401300E09
:1027F00082276EEC08F02EC182F40401300E82278D
:102800006EEC08F02FC182F40401300E82276EECCA
:1028100008F030C182F40401300E82276EEC08F01B
:1028200031C182F40401300E82276EEC08F032C10F
:1028300082F40401300E82276EEC08F033C182F47A
:102840000401300E82276EEC08F012002FC182F4D2
:102850000401300E82276EEC08F030C182F40401CE
:10286000300E82276EEC08F031C182F40401300E84
:1028700082276EEC08F032C182F40401300E822708
:102880006EEC08F033C182F40401300E82276EEC46
:1028900008F01200060E116E060E126E060E136E72
:1028A000112E50EF14F0122E50EF14F0132E50EFA3
:1028B00014F08B84020E116E020E126E020E136E55
:1028C000112E60EF14F0122E60EF14F0132E60EF53
:1028D00014F08B9412000101005305E1015303E150
:1028E000025301E1002B2EEC15F059EC16F0395192
:1028F000006F3A51016F420E046F4B0E056F000ED0
:10290000066F000E076F6FEC15F000C104F101C1F6
:1029100005F102C106F103C107F118C100F119C1A7
:1029200001F11AC102F11BC103F107B29CEF14F0CF
:1029300063EC15F09EEF14F05EEC15F000C118F199
:1029400001C119F102C11AF103C11BF1120059ECC6
:1029500016F059C100F15AC101F1060EA7EC06F0BC
:10296000E8CF04F1070EA7EC06F0E8CF05F1080E5A
:10297000A7EC06F0E8CF06F1090EA7EC06F0E8CFC9
:1029800007F15EEC15F000C124F101C125F102C18F
:1029900026F103C127F1290E046F000E056F000E0A
:1029A000066F000E076F6FEC15F0EE0E046F430E0E
:1029B000056F000E066F000E076F63EC15F024C163
:1029C00004F125C105F126C106F127C107F16FEC1D
:1029D00015F000C11CF101C11DF102C11EF103C1BE
:1029E0001FF1120EA7EC06F0E8CF04F1130EA7ECCE
:1029F00006F0E8CF05F1140EA7EC06F0E8CF06F1DB
:102A0000150EA7EC06F0E8CF07F10D0E006F000ED3
:102A1000016F000E026F000E036F6FEC15F0180EC1
:102A2000046F000E056F000E066F000E076F8FEC2F
:102A300015F01CC104F11DC105F11EC106F11FC135
:102A400007F163EC15F06A0E046F2A0E056F000E95
:102A5000066F000E076F5EEC15F01200BF0EFA6EE7
:102A6000200E3A6F396BD8900037013702370337A1
:102A7000D8B03FEF15F03A2F34EF15F039073A0789
:102A80000353D8B412000331070B80093F6F033999
:102A90000F0B010F396F80EC5FF0406F390580EC50
:102AA0005FF0405D405F396B3F33D8B03927393331
:102AB0003FA954EF15F040513927120001017EEC77
:102AC00016F0D8B01200010103510719346F41EC20
:102AD00016F0D8900751031934AF800F120001018E
:102AE000346B65EC16F0D8A07BEC16F0D8B0120071
:102AF00050EC16F059EC16F01F0E366F91EC16F0F4
:102B00000B35D8B041EC16F0D8A00335D8B0120080
:102B1000362F7EEF15F034B168EC16F0120001018B
:102B2000346B04510511061107110008D8A065EC9B
:102B300016F0D8A07BEC16F0D8B01200086B096B29
:102B40000A6B0B6B91EC16F01F0E366F91EC16F0C2
:102B500007510B5DD8A4B9EF15F006510A5DD8A452
:102B6000B9EF15F00551095DD8A4B9EF15F004517E
:102B7000085DD8A0CCEF15F00451085F0551D8A02E
:102B8000053D095F0651D8A0063D0A5F0751D8A050
:102B9000073D0B5FD8900081362FA6EF15F034B1BA
:102BA00068EC16F0346B65EC16F0D89095EC16F0E6
:102BB00007510B5DD8A4E9EF15F006510A5DD8A4C2
:102BC000E9EF15F00551095DD8A4E9EF15F00451BE
:102BD000085DD8A0F8EF15F0003FF8EF15F0013FC1
:102BE000F8EF15F0023FF8EF15F0032BD8B4120000
:102BF00034B168EC16F012000101346B65EC16F08C
:102C0000D8B012009AEC16F0200E366F003701375C
:102C10000237033711EE33F00A0E376FE7360A0E2C
:102C2000E75CD8B0E76EE552372F0EEF16F0362F7F
:102C300006EF16F034B12981D890120001010A0E76
:102C4000346F200E366F11EE29F03451376F0A0EB3
:102C5000D890E652D8B0E726E732372F29EF16F0A2
:102C60000333023301330033362F23EF16F0E750DE
:102C7000FF0FD8A00335D8B0120029B168EC16F0C8
:102C80001200045100270551D8B0053D0127065117
:102C9000D8B0063D02270751D8B0073D03271200E0
:102CA0000051086F0151096F02510A6F03510B6FF8
:102CB00012000101006B016B026B036B120001013A
:102CC000046B056B066B076B12000335D8A012006E
:102CD0000351800B001F011F021F031F003F78EFED
:102CE00016F0013F78EF16F0023F78EF16F0032B55
:102CF000342B032512000735D8A012000751800B92
:102D0000041F051F061F071F043F8EEF16F0053F27
:102D10008EEF16F0063F8EEF16F0072B342B0725AB
:102D200012000037013702370337083709370A37EF
:102D30000B3712000101296B2A6B2B6B2C6B2D6B4F
:102D40002E6B2F6B306B316B326B336B12000101CA
:102D50002A510F0B2A6F2B510F0B2B6F2C510F0B7E
:102D60002C6F2D510F0B2D6F2E510F0B2E6F2F51DE
:102D70000F0B2F6F30510F0B306F31510F0B316F25
:0E2D800032510F0B326F33510F0B336F1200B5
:10BF0000E844F926000C160C2B0C3F0C520C640C68
:10BF1000760C860C960CA50CB30CC10CCF0CDC0C6B
:06BF2000E80CF40C000C1B
:00000001FF
